:020000040800F2
:1000000000000220BD220008E1200008E3200008D3
:10001000E5200008E7200008E920000800000000B3
:10002000000000000000000000000000EB200008BD
:10003000ED20000800000000EF200008F12000087B
:100040000D2300080D2300080D2300080D230008D0
:100050000D2300080D2300080D2300080D230008C0
:100060000D2300080D2300080D2300080D230008B0
:100070000D2300080D2300080D2300080D230008A0
:100080000D2300080D2300080D2300080D23000890
:100090000D2300080D2300080D2300080D23000880
:1000A0000D2300080D2300080D2300080D23000870
:1000B0000D230008412200080D2300080D2300082D
:1000C0000D2300080D2300080D2300080D23000850
:1000D0000D2300080D230008512200080D230008FD
:1000E0000D2300080D2300080D2300080D23000830
:1000F0000D2300080D2300080D2300080D23000820
:100100000D2300080D2300080D2300080D2300080F
:100110000D2300080D2300080D2300080D230008FF
:100120000D2300080D2300080D2300080D230008EF
:100130000D23000800000000000000000D2300084F
:100140000D2300080D2300080D2300080D230008CF
:100150000D2300080D2300080D2300080D230008BF
:100160000D2300080D2300080D2300080D230008AF
:100170000D2300080D2300080D23000800000000D7
:10018000000000000D230008000000000000000037
:100190000D23000800000000000000000D230008EF
:1001A0000000000000000000000000000D23000817
:1001B0000D2300080D2300080D2300080D2300085F
:0401C0000D23000803
:1001C40010B5054C237833B9044B13B10448AFF38D
:1001D40000800123237010BDF00100200000000006
:1001E4008825000808B5034B1BB103490348AFF346
:1001F400008008BD00000000F401002088250008EC
:1002040053B94AB9002908BF00281CBF4FF0FF3179
:100214004FF0FF3000F072B9ADF1080C6DE904CE77
:1002240000F006F8DDF804E0DDE9022304B07047CD
:100234002DE9F047089E04468846002B4BD18A429C
:10024400154667D9B2FA82F24AB1C2F1200701FA1F
:1002540002F320FA07F7954047EA030894404FEA6F
:10026400154E230CB8FBFEF71FFA85FC0EFB17880E
:1002740043EA084307FB0CF1994209D9EB1807F14B
:10028400FF3080F01B81994240F21881023F2B44D9
:100294005B1AA4B2B3FBFEF00EFB103344EA034432
:1002A40000FB0CFCA44509D92C1900F1FF3380F0A4
:1002B4000781A44540F2048102382C4440EA0740F7
:1002C400A4EB0C0400271EB1D4400023C6E900436C
:1002D4003946BDE8F0878B4209D9002E00F0EB8047
:1002E4000027C6E9000138463946BDE8F087B3FA6D
:1002F40083F7002F47D18B4202D3824200F2FA8067
:10030400841A61EB030301209846002EE0D0C6E96D
:100314000048DDE702B9FFDEB2FA82F2002A40F0BB
:100324008F80491B4FEA154E1FFA85F80127B1FB50
:10033400FEFC230C0EFB1C1143EA014308FB0CF1E9
:10034400994207D9EB180CF1FF3002D2994200F21E
:10035400CD808446591AA3B2B1FBFEF00EFB1014F3
:1003640043EA044408FB00F8A04507D92C1900F11E
:10037400FF3302D2A04500F2B6801846A4EB08046D
:1003840040EA0C409FE7C7F1200CBB4022FA0CFE68
:100394004EEA030E01FA07F420FA0CF521FA0CF3E5
:1003A4004FEA1E482543B3FBF8F92C0C08FB19331C
:1003B4001FFA8EFA44EA034309FB0AF49C4202FA48
:1003C40007F200FA07F10BD91EEB030309F1FF3022
:1003D40080F087809C4240F28480A9F10209734432
:1003E4001B1BADB2B3FBF8F008FB103345EA034422
:1003F40000FB0AFAA24508D91EEB040400F1FF33FE
:100404006BD2A24569D90238744440EA0940A0FB82
:100414000289A4EB0A044C45C2464B4654D351D03E
:10042400002E69D0B1EB0A0564EB030404FA0CFC5A
:10043400FD40FC404CEA0505C6E90054002747E7A7
:10044400C2F1200320FA03F7954001FA02F021FAE1
:1004540003F34FEA154E3843010CB3FBFEF71FFAC2
:1004640085F80EFB173341EA034107FB08F38B427F
:1004740004FA02F407D9691807F1FF3C2FD28B4222
:100484002DD9023F2944CB1A81B2B3FBFEF00EFBF7
:10049400103341EA034100FB08F38B4207D9691882
:1004A40000F1FF3C17D28B4215D902382944C91AEE
:1004B40040EA07473BE73746304609E70746E7E6A1
:1004C4001846FBE64145ABD2B8EB020A69EB0E02D3
:1004D40001381346A4E76046E9E7184695E76746FE
:1004E400D1E781467CE702382C4447E7ACF1020CA3
:1004F4002B442FE7384608E73746E9E6704700BF44
:1005040010B504460E4B18784FF47A73B3FBF0F32E
:100514000C4A1068B0FBF3F000F0A8F868B90F2C8F
:1005240001D901200AE0002221464FF0FF3000F0FB
:100534005DF8034B5C60002000E0012010BD00BFAB
:10054400000000201C00002008B50B4B1A6842F480
:1005540000721A601A6842F480621A601A6842F4DF
:1005640080721A60032000F02FF80020FFF7C8FF04
:1005740001F0D4FC002008BD003C0240034A11688D
:10058400034B1B780B441360704700BF1802002014
:1005940000000020014B1868704700BF18020020BB
:1005A40038B50446FFF7F6FF0546B4F1FF3F02D025
:1005B400044B1B781C44FFF7EDFF401BA042FAD309
:1005C40038BD00BF00000020074AD36823F4E0636D
:1005D4001B041B0C000200F4E060184340F0BF60F1
:1005E40040F40030D060704700ED00E030B4174BA9
:1005F400DB68C3F30223C3F10704042C28BF0424DB
:100604001D1D062D18D9033B4FF0FF3505FA04F4E0
:1006140021EA0401994005FA03F322EA030319438A
:1006240000280BDB0901C9B200F1604000F561400C
:1006340080F8001330BC70470023E5E700F00F009A
:100644000901C9B2024B1954F4E700BF00ED00E000
:1006540014ED00E000F01F02400901239340024A18
:1006640042F82030704700BF00E100E00138B0F1EB
:10067400807F0AD2064B5860064AF02182F8231084
:100684000020986007221A6070470120704700BF5D
:1006940010E000E000ED00E090F83530DBB2022B12
:1006A40003D08023436501207047052380F835304B
:1006B4000268136823F001031360002070470000F0
:1006C40000230F2B00F2D180F0B482B039E006226F
:1006D40000E00022B2403A430234644E46F824203B
:1006E400634A1468EA4302EA04064F6817F4803F39
:1006F40001D045EA04065E4C2660646802EA0406FA
:100704004F6817F4003F01D045EA0406584C666070
:10071400A46802EA04064F6817F4801F01D045EA72
:100724000406534CA660E46822404E6816F4001F89
:1007340001D045EA04024E4CE26001330F2B00F273
:10074400918001229A400C6804EA0205AA42F4D17D
:100754004C68022C01D0122C10D1DE08083650F857
:1007640026C003F00704A7000F24BC402CEA040CA5
:100774000C69BC4044EA0C0440F8264004685F005D
:100784000326BE40F64306EA040C4C6804F0030456
:10079400BC4044EA0C0404604C6804F1FF3CBCF126
:1007A400010F03D9112C01D0122C10D1846806EA50
:1007B400040CCC68BC4044EA0C048460446824EA19
:1007C40002024C68C4F300149C4014434460C268A1
:1007D40016408A68BA403243C2604A6812F0805FA9
:1007E400ABD000220192234A546C44F480445464F4
:1007F400526C02F480420192019A9C08A61C1B4A86
:1008040052F8267003F0030296000F22B24027EA42
:100814000207194A90423FF45CAF02F580629042AD
:1008240016D002F58062904214D002F580629042A4
:1008340012D002F58062904210D002F5806290429C
:100844000ED002F5806290423FF441AF072241E7A7
:1008540001223FE702223DE703223BE7042239E776
:10086400052237E702B0F0BC7047704700380140FA
:10087400003C0140003802400000024010B582B044
:1008840000230193194B1A6C42F080521A641B6CBA
:1008940003F080530193019B154B01221A60FFF76B
:1008A40079FE0446134B5B6813F4803F08D1FFF7CD
:1008B40071FE001BB0F57A7FF4D9032002B010BD9D
:1008C4000D4B01221A60FFF765FE0446094B5B6875
:1008D40013F4003F07D1FFF75DFE001BB0F57A7FEC
:1008E400F4D90320EAE70020E8E700BF003802401B
:1008F40040000E420070004044000E42002800F008
:100904009D8070B504464F4B1B6803F00F038B4268
:1009140009D2CBB24B4A1370136803F00F038B4216
:1009240001D0012070BD236813F0020F17D013F01B
:10093400040F04D0444A936843F4E053936023685B
:1009440013F0080F04D0404A936843F46043936063
:100954003D4A936823F0F003A068034393600D4677
:10096400236813F0010F32D06368012B21D09A1E43
:10097400012A25D9344A126812F0020F60D0324994
:100984008A6822F0030213438B60FFF703FE0646D6
:100994002D4B9B6803F00C036268B3EB820F16D0F7
:1009A400FFF7F8FD801B41F288339842F0D9032009
:1009B400B8E7254A126812F4003FE0D10120B1E7FC
:1009C400214A126812F0007FD9D10120AAE71D4BF9
:1009D4001B6803F00F03AB4209D9EAB2194B1A7032
:1009E4001B6803F00F03AB4201D001209AE7236890
:1009F40013F0040F06D0144A936823F4E053E1681B
:100A04000B439360236813F0080F07D00E4A9368D2
:100A140023F46043216943EAC103936000F040F882
:100A2400094B9B68C3F30313084AD35CD840084BB3
:100A340018600020FFF764FD002073E70120704771
:100A440001206FE7003C024000380240A025000866
:100A54001C000020014B1868704700BF1C000020D8
:100A640008B5FFF7F7FF044B9B68C3F38223034ADF
:100A7400D35CD84008BD00BF00380240B025000850
:100A840008B5FFF7E7FF044B9B68C3F34233034AFF
:100A9400D35CD84008BD00BF00380240B025000830
:100AA4002DE9F04B5C4B9B6803F00C03082B07D03B
:100AB4000C2B5BD0042B00F0AD805848BDE8F08BC4
:100AC400554B5A6802F03F025B6813F4800F2AD03A
:100AD400514B5B68C3F388131E4600275C01002555
:100AE400E41A65EB0705A90141EA9461A001001B22
:100AF40061EB0501CB0043EA5073C400A01943EB3A
:100B040007014B0243EAD05344022046194600230E
:100B1400FFF776FB404B5B68C3F3014301335B0093
:100B2400B0FBF3F0CAE73C4B5B68C3F388131E4683
:100B340000275C010025E41A65EB0705A90141EAD9
:100B44009461A001001B61EB0501CB0043EA5073E3
:100B5400C400A01943EB07018B0243EA90538402BB
:100B6400204619460023FFF74BFBD3E72A4B5A686C
:100B740002F03F025B6813F4800F28D0264B5B68B9
:100B8400C3F388131E4600275C010025E41A65EBB5
:100B94000705A90141EA9461A001001B61EB05016D
:100BA400CB0043EA5073C400A01943EB07014B0286
:100BB40043EAD0534402204619460023FFF720FBA2
:100BC400154B5B68C3F30273B0FBF3F076E7124B8B
:100BD4005B68C3F388131E4600275C010025E41AF2
:100BE40065EB0705A90141EA9461A001001B61EBD3
:100BF4000501CB0043EA5073C400A01943EB07017D
:100C04008B0243EA90538402204619460023FFF7DF
:100C1400F7FAD5E7024851E7003802400024F4000F
:100C240000127A0070B582B00446036813F0010F15
:100C340041D0A64B9B6803F00C03042B32D0A34B8A
:100C44009B6803F00C03082B27D0A04B9B6803F090
:100C54000C030C2B59D06368B3F5803F5BD0B3F51C
:100C6400A02F5ED0994B1A6822F480321A601A6859
:100C740022F480221A606368002B5CD0FFF78AFCA0
:100C84000546924B1B6813F4003F14D1FFF782FC16
:100C9400401B6428F5D903209DE18C4B5B6813F459
:100CA400800FD2D0894B1B6813F4003F03D06368D4
:100CB400002B00F08D81236813F0020F67D0834B63
:100CC4009B6813F00C0F4AD0804B9B6803F00C0315
:100CD400082B3FD07D4B9B6803F00C030C2B48D0B2
:100CE400E368002B74D07A4B01221A60FFF752FCA0
:100CF4000546764B1B6813F0020F60D1FFF74AFCE0
:100D0400401B0228F5D9032065E1704B5B6813F49E
:100D1400800FA0D0C6E76D4A136843F48033136094
:100D2400A9E76A4B1A6842F480221A601A6842F4EE
:100D340080321A609FE7FFF72DFC0546634B1B6862
:100D440013F4003FB7D0FFF725FC401B6428F5D906
:100D5400032040E15D4B5B6813F4800FBAD15B4B19
:100D64001B6813F0020F0AD0E368012B07D001209F
:100D740031E1564B5B6813F4800FB1D1EFE7534A6E
:100D8400136823F0F803216943EAC103136023685D
:100D940013F0080F40D0636963B34E4B01221A600D
:100DA400FFF7F8FB0546494B5B6F13F0020F33D195
:100DB400FFF7F0FB401B0228F5D903200BE1434A5F
:100DC400136823F0F803216943EAC1031360DEE7E3
:100DD4003F4B00221A60FFF7DDFB05463B4B1B68C7
:100DE40013F0020FD3D0FFF7D5FB401B0228F5D92F
:100DF4000320F0E0374B00221A60FFF7CBFB0546D7
:100E0400324B5B6F13F0020F06D0FFF7C3FB401B9E
:100E14000228F5D90320DEE0236813F0040F79D00B
:100E24002A4B1B6C13F0805F33D100230193274BB3
:100E34001A6C42F080521A641B6C03F080530193C5
:100E4400019B0125244B1B6813F4807F23D0A368E6
:100E5400012B34D0052B41D01C4B1A6F22F0010218
:100E64001A671A6F22F004021A67A368002B3FD096
:100E7400FFF790FB0646154B1B6F13F0020F48D18A
:100E8400FFF788FB801B41F288339842F3D9032093
:100E9400A1E00025D6E7104A136843F48073136079
:100EA400FFF778FB06460C4B1B6813F4807FCED10A
:100EB400FFF770FB801B0228F5D903208BE0034A5F
:100EC400136F43F001031367CFE700BF00380240FC
:100ED40000004742800E474200700040404B1A6FAA
:100EE40042F004021A671A6F42F001021A67BCE763
:100EF400FFF750FB06463A4B1B6F13F0020F08D066
:100F0400FFF748FB801B41F288339842F3D9032052
:100F140061E0E5B9A369002B5CD0314A926802F024
:100F24000C02082A59D0022B17D02E4B00221A602B
:100F3400FFF730FB04462A4B1B6813F0007F45D0B3
:100F4400FFF728FB001B0228F5D9032043E0244ABD
:100F5400136C23F080531364DCE7224B00221A60E5
:100F6400FFF718FB05461E4B1B6813F0007F06D0E5
:100F7400FFF710FB401B0228F5D903202BE0E3699F
:100F8400226A1343626A43EA8213A26A5208013A4C
:100F940043EA0243E26A43EA0263226B43EA0273CE
:100FA4000F4A53600F4B01221A60FFF7F3FA04460D
:100FB4000B4B1B6813F0007F06D1FFF7EBFA001B05
:100FC4000228F5D9032006E0002004E0002002E016
:100FD400012000E0002002B070BD0120FBE700BF4B
:100FE400003802406000474270B4036A23F00103F2
:100FF4000362036A4268846924F073040D6845EA55
:10100400040623F002048B6823430C4DA84202D04B
:101014000B4CA0420BD123F00803CD682B4323F0E3
:10102400040322F440724D6915438A692A434260DD
:1010340086614A684263036270BC704700000140E5
:101044000004014030B4036A23F480730362036A2A
:101054004268C46924F073040D682C4323F40073BC
:101064008D6843EA05230E4DA84203D005F580653B
:10107400A8420ED123F40063CD6843EA052323F488
:10108400806322F440524D6942EA05128D6942EAB6
:1010940005124260C4614A68C263036230BC70478F
:1010A4000000014030B4036A23F480530362036AEE
:1010B4004468C26922F4E6420D6842EA052223F438
:1010C40000538D6843EA0533094DA84203D005F562
:1010D4008065A84204D124F480444D6944EA85140F
:1010E4004460C2614A680264036230BC704700BF56
:1010F400000001407047704770477047704710B553
:10110400044603681A6912F0020F11D0DA6812F06B
:10111400020F0DD06FF002021A61012303760368F7
:101124009B6913F0030F70D0FFF7E6FF00232376CB
:1011340023681A6912F0040F12D0DA6812F0040F4F
:101144000ED06FF004021A610223237623689B6990
:1011540013F4407F5FD02046FFF7CEFF00232376B1
:1011640023681A6912F0080F12D0DA6812F0080F17
:101174000ED06FF008021A61042323762368DB691A
:1011840013F0030F4ED02046FFF7B6FF002323765B
:1011940023681A6912F0100F12D0DA6812F0100FD7
:1011A4000ED06FF010021A61082323762368DB69DE
:1011B40013F4407F3DD02046FFF79EFF00232376A3
:1011C40023681A6912F0010F03D0DA6812F0010FD4
:1011D40036D123681A6912F0800F03D0DA6812F04E
:1011E400800F34D123681A6912F0400F03D0DA68F3
:1011F40012F0400F32D123681A6912F0200F03D085
:10120400DA6812F0200F30D110BDFFF774FF2046CA
:10121400FFF773FF8AE72046FFF76DFF2046FFF7CD
:101224006CFF9BE72046FFF766FF2046FFF765FF4C
:10123400ACE72046FFF75FFF2046FFF75EFFBDE700
:101244006FF001021A612046FFF754FFC1E76FF007
:1012540080021A61204600F0EDF9C3E76FF0400206
:101264001A612046FFF74AFFC5E76FF020021A61B2
:10127400204600F0DEF9C7E703682E4A904212D0F8
:10128400B0F1804F0FD0A2F57C4290420BD002F512
:101294008062904207D002F58062904203D002F54A
:1012A4007842904203D123F070034A681343214AE1
:1012B40090422AD0B0F1804F27D0A2F57C429042D0
:1012C40023D002F5806290421FD002F580629042E2
:1012D4001BD002F57842904217D002F5705290422A
:1012E40013D002F5806290420FD002F580629042E2
:1012F4000BD0A2F59832904207D002F5806290425A
:1013040003D002F58062904203D123F44073CA688B
:10131400134303608B68C3620B688362054B984276
:1013240003D003F58063984201D10B690363012361
:101334004361704700000140A8B110B5044690F81D
:1013440039305BB1022384F83930211D2068FFF75E
:1013540093FF012384F83930002010BD80F8383021
:1013640000F030FEEEE701207047002847D0F8B5C2
:1013740005460C4690F83930002B3BD0022385F803
:101384003930294651F8042B936823F007039360FE
:101394002868FFF771FF29688A688E690F6A2068D8
:1013A400104326F4407626F00306A268A36942EAB5
:1013B4000323334323F47C4323F0FC03E668E2690C
:1013C40046EA02261E43226A1303226943EA0213F1
:1013D400334327F0AA076268646942EA04123A4375
:1013E400886029688B612B681A62012385F839307B
:1013F4000020F8BD80F8383000F0B0FDBEE70120D1
:101404007047000030B4036A23F010030362036AD8
:101414004468826922F4E6420D6842EA052223F018
:1014240020038D6843EA05130E4DA84203D005F549
:101434008065A8420ED123F08003CD6843EA0513EA
:1014440023F0400324F440644D6944EA85048D6923
:1014540044EA8504446082614A688263036230BC62
:10146400704700BF0000014038B590F83830012BB8
:1014740066D00D460446012380F83830022380F8F4
:1014840039300C2A1AD8DFE802F007191919201983
:1014940019193419191947000068FFF7A5FD2268C6
:1014A400936943F0080393612268936923F004036A
:1014B40093612268936929690B439361012384F83A
:1014C4003930002084F8380038BD0068FFF79AFFEF
:1014D4002268936943F4006393612268936923F457
:1014E4008063936122689369296943EA01239361C4
:1014F400E4E70068FFF7A6FD2268D36943F0080318
:10150400D3612268D36923F00403D3612268D369C9
:1015140029690B43D361D1E70068FFF7C3FD226853
:10152400D36943F40063D3612268D36923F48063ED
:10153400D3612268D369296943EA0123D361BDE7F2
:101544000220C1E710B4012303FA01F4036A23EA79
:1015540004030362036A8A40134303625DF8044B85
:101564007047000010B5044601220068FFF7EAFF47
:101574002368094A934203D002F58062934203D15F
:101584005A6C42F400425A642268136843F001031F
:101594001360002010BD00BF0000014010B50446D8
:1015A40061B1042916D0012200210068FFF7CAFFA7
:1015B400012204212068FFF7C5FF04E00122002175
:1015C4000068FFF7BFFF2268136843F0010313604C
:1015D400002010BD012204210068FFF7B3FFF2E7E9
:1015E40090F83830012B22D030B4012280F8382012
:1015F400022380F839300468636823F07003636061
:10160400046863680D682B4363600468A36823F06F
:101614008003A3600468A36849680B43A36080F84F
:101624003920002380F83830184630BC7047022037
:101634007047704770470268D36823F49073D3608F
:101644000268536923F001035361202380F83A3080
:10165400704790F83930DBB2212B2AD18368B3F577
:10166400805F16D0036A5A1C02621A7803685A60B3
:10167400C38C013B9BB2C384EBB90268D36823F0EB
:101684008003D3600268D36843F04003D360002032
:101694007047036A1B880268C3F308035360036935
:1016A4001BB9036A02330362E2E7036A013303628C
:1016B400DEE7022070470020704700002DE9F84360
:1016C400044601680A6922F44052C36813430B615B
:1016D4000168CA6822F4164222F00C028368006989
:1016E400034360690343E06903431343CB60216808
:1016F4004A6922F44072A36913434B61E369B3F569
:10170400004F60D02368B84A934200F0148102F578
:101714008062934200F00F81FFF7A2F900EB800092
:1017240000EB80006568AD00B0FBF5F5AF4FA7FB9B
:1017340005356D092E01FFF793F900EB800000EBEE
:1017440080006568AD00B0FBF5F9FFF789F900EB9F
:10175400800000EB80006568AD00B0FBF5F5A7FBE9
:1017640005356D094FF0640808FB15952D013235D8
:10177400A7FB05356D0905F0F0053544FFF770F951
:1017840000EB800000EB80006668B600B0FBF6F664
:10179400FFF766F900EB800000EB800063689B00B4
:1017A400B0FBF3F0A7FB0030400908FB10684FEAD8
:1017B400081808F13208A7FB0837C7F34317236852
:1017C4002F449F600DE12368874A93425BD002F562
:1017D4008062934257D0FFF743F900EB800000EB9F
:1017E400800065686D00B0FBF5F5804FA7FB0535FB
:1017F4006D092E01FFF734F900EB800000EB800047
:1018040065686D00B0FBF5F9FFF72AF900EB80007D
:1018140000EB800065686D00B0FBF5F5A7FB0535AE
:101824006D094FF0640808FB1595ED003235A7FBF0
:1018340005356D096D0005F4F8753544FFF710F9A9
:1018440000EB800000EB800066687600B0FBF6F6E3
:10185400FFF706F900EB800000EB800063685B0093
:10186400B0FBF3F3A7FB03235B0908FB13684FEA00
:10187400C80808F13208A7FB0837C7F342172368E2
:101884002F449F60ADE0FFF7FBF800EB800000EB16
:10189400800065686D00B0FBF5F5544FA7FB053576
:1018A4006D092E01FFF7ECF800EB800000EB8000DF
:1018B40065686D00B0FBF5F9FFF7E2F800EB800016
:1018C40000EB800065686D00B0FBF5F5A7FB0535FE
:1018D4006D094FF0640808FB1595ED003235A7FB40
:1018E40005356D096D0005F4F8753544FFF7C8F842
:1018F40000EB800000EB800066687600B0FBF6F633
:10190400FFF7BEF800EB800000EB800063685B002B
:10191400B0FBF3F3A7FB03235B0908FB13684FEA4F
:10192400C80808F13208A7FB0837C7F34217236831
:101934002F449F6055E0FFF7A3F800EB800000EB15
:1019440080006568AD00B0FBF5F5284FA7FB0535B1
:101954006D092E01FFF794F800EB800000EB800086
:101964006568AD00B0FBF5F9FFF78AF800EB80007D
:1019740000EB80006568AD00B0FBF5F5A7FB05350D
:101984006D094FF0640808FB15952D013235A7FB4E
:1019940005356D0905F0F0053544FFF771F800EBE6
:1019A400800000EB80006668B600B0FBF6F6FFF737
:1019B40067F800EB800000EB800063689B00B0FBDD
:1019C400F3F0A7FB0030400908FB10684FEA081841
:1019D40008F13208A7FB0837C7F3431723682F44DD
:1019E4009F60BDE8F88300BF001001401F85EB51E4
:1019F40058B310B5044690F839300BB3242384F857
:101A040039302268D36823F40053D3602046FFF7AB
:101A140055FE2268136923F49043136122685369C5
:101A240023F02A0353612268D36843F40053D3603C
:101A34000020E063202384F8393084F83A3010BD64
:101A440080F8383000F00AFBD8E70120704790F89E
:101A54003930DBB2202B16D1B9B1C2B190F838308D
:101A6400012B16D001628284C2840023C363212225
:101A740080F8392080F838300168CA6842F0800262
:101A8400CA60184670470220704701207047012041
:101A940070470220704790F83A30DBB2202B1BD1FC
:101AA400E1B1EAB190F83830012B1BD08162828514
:101AB400C2850023C363222280F83A2080F838309C
:101AC40001684A6942F001024A610168CA6842F445
:101AD4009072CA6018467047022070470120704710
:101AE4000120704702207047704708B50168CB6831
:101AF40023F04003CB60202380F83930FFF7F4FF54
:101B0400002008BD704708B590F83A30DBB2222BAC
:101B140040D18368B3F5805F0ED0036903BB0368CB
:101B24005A68836A591C81621A70C38D013B9BB247
:101B3400C385F3B100202EE0826A036943B90368C8
:101B44005B68C3F308031380836A02338362ECE7A0
:101B540003685B68DBB21380836A01338362E4E762
:101B640003685B68826A511C816203F07F0313700F
:101B7400DBE70268D36823F49073D3600268536987
:101B840023F001035361202380F83A30FFF7BAFFB2
:101B9400002000E0022008BD7047000010B5044694
:101BA40002681368D168526913F00F0005D113F06D
:101BB400200F02D011F0200F53D1002867D012F06B
:101BC400010202D111F4907F61D013F0010F06D00D
:101BD40011F4807F03D0E06B40F00100E06313F068
:101BE400040F04D01AB1E06B40F00200E06313F07C
:101BF400020F04D01AB1E06B40F00400E06313F06C
:101C0400080F04D01AB1E26B42F00802E263E26BFF
:101C1400002A48D013F0200F02D011F0200F24D155
:101C240023685B6903F04003E26B12F0080F00D1F4
:101C34003BB32046FFF7FFFC23685A6912F0400FBC
:101C44001BD05A6922F040025A61636B8BB11A4A65
:101C54001A65606BFEF720FD28B3606B036D98472F
:101C640021E02046FFF74FFF1DE02046FFF74BFF22
:101C7400D6E72046FFF790FF15E02046FFF78CFFDC
:101C840011E02046FFF788FF0023E3630BE013F025
:101C9400800F02D011F0800F06D113F0400F02D054
:101CA40011F0400F04D110BD2046FFF7D2FCFAE733
:101CB4002046FFF71AFFF6E7C11C000808B5806B41
:101CC4000023C385C384FFF767FF08BD82B00023E8
:101CD4000193064B1A6B42F001021A631B6B03F06B
:101CE40001030193019B02B0704700BF003802401A
:101CF40008B50848084B03604FF4E1334360002300
:101D04008360C36003610C2242618361C361FFF796
:101D14006FFE08BD9C0200200044004030B58DB029
:101D24002022002104A800F033FB00250195029530
:101D34000C4C4FF0804323606560A5604FF0FF3387
:101D4400E3602561012303930593099303A92046C6
:101D5400FFF70BFB0195029501A92046FFF740FC14
:101D64000DB030BD6002002030B58BB00024089463
:101D7400099401940294039404940594069407949A
:101D8400134D144B2B606C60AC604FF6FF73EB602B
:101D94002C612846FFF7D0FA0894099408A928462C
:101DA400FFF71EFC602301930294039405942246DA
:101DB40001A92846FFF758FB04220DEB020128462F
:101DC400FFF752FB284600F01DF90BB030BD00BFF1
:101DD400200200200004004030B595B034220021D8
:101DE40007A800F0D5FA00240294039404940594FF
:101DF400069400941C4B1A6C42F080521A641B6CBB
:101E040003F080530093009B0194184B1A6842F42A
:101E140040421A601B6803F440430193019B02256E
:101E2400079501230A9310230B930D950E94082311
:101E34000F93B423109311951295139507A8FEF7E9
:101E4400F1FEFEF71BFD0F230293039504944FF458
:101E5400A05305934FF480530693052102A8FEF77F
:101E64004DFD15B030BD00BF003802400070004089
:101E740000B585B0FEF768FBFFF7AEFFFFF726FF5E
:101E8400FFF736FFFFF74AFFFFF76EFF00240194C8
:101E94000294ADF80C40124D21462846FFF762FB30
:101EA40004212846FFF75EFB0E4B5C639C630E4DDA
:101EB40004212846FFF772FB21462846FFF76EFBF4
:101EC4000A2201A9094B186800F060FA0A2201A944
:101ED4000748FFF7BCFD4FF47A70FEF761FBEFE7AC
:101EE4002002002000040040600200205C02002068
:101EF4009C020020002807DB0028B8BF4042064BA4
:101F0400586300229A637047034B00225A630028E7
:101F1400B8BF4042986370470004004000B583B0E6
:101F2400002100910C4B5A6C42F480425A645A6C62
:101F340002F480420092009A01911A6C42F080529D
:101F44001A641B6C03F080530193019B0720FEF776
:101F54003BFB03B05DF804FB0038024000B589B0D8
:101F64000023039304930593069307930368B3F143
:101F7400804F02D009B05DF804FB0021019103F504
:101F84000E331A6C42F001021A641A6C02F0010258
:101F94000192019A02911A6B42F001021A631B6BBF
:101FA40003F001030293029B03230393022304938C
:101FB40001230593079303A90148FEF781FBD9E7A1
:101FC4000000024002680E4B9A4200D0704700B5F0
:101FD40083B00021019103F50D331A6C42F0020223
:101FE4001A641B6C03F002030193019B0A461D2033
:101FF400FEF7FCFA1D20FEF72DFB03B05DF804FB91
:102004000004004000B587B00023019302930393BA
:102014000493059302680E4B9A4202D007B05DF810
:1020240004FB002300930B4B1A6B42F001021A636A
:102034001B6B03F001030093009BC0230193022355
:102044000293059301A90448FEF73AFBE6E700BFB3
:1020540000040040003802400000024010B588B07F
:102064000023039304930593069307930268194B83
:102074009A4201D008B010BD0024019403F5FA334C
:102084001A6C42F400321A641A6C02F4003201929F
:10209400019A02941A6B42F001021A631B6B03F05B
:1020A40001030293029B0C23039302230493012351
:1020B4000593032306930723079303A90648FEF712
:1020C400FFFA224621462620FEF790FA2620FEF744
:1020D400C1FACFE700440040000002407047FEE729
:1020E400FEE7FEE7FEE770477047704770B5FEF7FE
:1020F40045FA4FF080435B6A444D2B600622444905
:102104004448FFF7C8FC444C63682360A3682A680A
:102114009B1A6360414D424E33682B60FEF73AFAD6
:1021240030602B68C01A3F4B1860626807EE902A33
:10213400F8EEE77A3C4D95ED007A67EE877AFDEE8E
:10214400E77A17EE901A394BC3ED007A2368D41A54
:1021540007EE104AB8EEC77AD5ED017A27EE277A52
:1021640007EE900AF8EEE77AC7EE276ABDEEE67A44
:1021740017EE100A2E4C84ED007AD31807EE103AAD
:10218400B8EEC77AD5ED026A27EE267A67EE877A2B
:10219400B6EE007A67EE877A264A92ED007AB8EEB8
:1021A400C77A77EE277AFDEEE77A17EE903AC2ED1A
:1021B400007A01440B44204A1360EA6893420BDC22
:1021C40051428B4214DB8B421BDC93420BDA164BDD
:1021D4004FF07E529A6006E0174B1A600022AA6004
:1021E400144B00221A60144B1868FFF783FE70BD6D
:1021F400114B19600C4B00229A600E4B00221A609E
:10220400F1E7094B4FF07E529A60ECE75C02002044
:10221400080000209C0200200C020020DC020020A8
:10222400E4020020F00200200C000020EC02002058
:10223400E8020020E0020020F402002008B5024871
:10224400FEF75DFF08BD00BF2002002008B504486A
:10225400FFF7A4FC034800F058F8034B986008BD4E
:102264009C020020080000200C0200200F49D1F835
:10227400883043F47003C1F888300D4B1A6842F07B
:1022840001021A60002098601A6822F0847222F415
:1022940080321A60074A5A601A6822F480221A604F
:1022A400D8604FF000638B60704700BF00ED00E022
:1022B4000038024010300024DFF834D0002103E05D
:1022C4000C4B5B58435004310B480C4B42189A4258
:1022D400F6D30B4A02E0002342F8043B094B9A422E
:1022E400F9D3FFF7C3FF00F015F8FFF7C1FD7047FE
:1022F40000000220F826000800000020F001002061
:10230400F0010020F8020020FEE70A22002100F07C
:10231400C3B8000070B50D4E0D4CA41BA4100025CD
:10232400A54209D10B4E0C4C00F02CF9A41BA410AF
:102334000025A54205D170BD56F8253098470135D2
:10234400EEE756F8253098470135F2E7F026000805
:10235400F0260008F0260008F4260008931E222B1D
:1023640010B50C4604D900230B701C46204610BD42
:102374000A2A09D1002807DA2D230B7040420121D3
:10238400214400F09FF8F1E70021F9E7FFF7E6BFE9
:1023940002440346934200D1704703F8011BF9E756
:1023A4002DE9F0478046894692461E460F463D4633
:1023B400089815F8014B00F0C3F82044437813F053
:1023C400080332D12D2C32D17C78BD1C0122002E81
:1023D4005DD0102E09D1302C07D12B7803F0DF0308
:1023E400582B4FD16C7810260235002A14BF4FF0B9
:1023F40000416FF000410027B1FBF6FC384606FBB4
:102404001C1EA4F13003092B17D81C46A64223DD59
:102414007B1C07D084451CD301D1A64519DB00FBE6
:102424000640012715F8014BEBE72F46BFE72B2C9D
:1024340004BFBD1C7C781A46C9E7A4F14103192BDB
:1024440001D8373CE2E7A4F16103192B04D8573CC7
:10245400DCE74FF0FF37E5E77B1C08D12223C8F8FF
:1024640000300846BAF1000F07D1BDE8F08702B189
:102474004042BAF1000FF8D00FB105F1FF39CAF8A4
:102484000090F2E73024002EAFD10826ADE7302CBF
:10249400A3D00A26A9E70000084B37B51C68084DED
:1024A400236A002B08BF2B46009313460A460146B5
:1024B4002046FFF775FF03B030BD00BF20000020A9
:1024C40084000020F0B51D4B8BB005460C466E46CB
:1024D40003F1200C18685968374603C7083363456D
:1024E4003E46F7D118681B793B71931E222B386046
:1024F4004FF0000304D923701C4620460BB0F0BDF6
:10250400661EB5FBF2F00AAF02FB10553D44591CA0
:1025140015F8285C06F8015F054668B96054234441
:102524002246191B101B8142E7DD1178187802F846
:10253400010B03F80119F4E70B46E2E7B82500089C
:10254400D0F8EC00704782B001B901A942B14BB197
:1025540013780B601278101C18BF012002B070476A
:102564001046FBE76FF00100F8E749B1FF2A85BF89
:102574008A2303600A704FF0FF3098BF0120704730
:1025840008467047F8B500BFF8BC08BC9E467047C3
:0C259400F8B500BFF8BC08BC9E467047BC
:1025A0000000000000000000010203040607080903
:1025B0000000000001020304303132333435363775
:1025C00038396162636465666768696A6B6C6D6EF1
:1025D0006F707172737475767778797A00430050F2
:1025E0004F534958002E000020202020202020207A
:1025F00020282828282820202020202020202020B3
:1026000020202020202020208810101010101010D2
:10261000101010101010101004040404040404041A
:1026200004041010101010101041414141414101AB
:10263000010101010101010101010101010101018A
:102640000101011010101010104242424242420299
:10265000020202020202020202020202020202025A
:102660000202021010101020000000000000000004
:10267000000000000000000000000000000000005A
:10268000000000000000000000000000000000004A
:10269000000000000000000000000000000000003A
:1026A000000000000000000000000000000000002A
:1026B000000000000000000000000000000000001A
:1026C000000000000000000000000000000000000A
:1026D00000000000000000000000000000000000FA
:0826E0000000000000000000F2
:0826E8004CDBFF7F0100000044
:0426F000E9010008F4
:0426F400C501000814
:1026F8000100000010000000300000000000484405
:102708000060EA460000803F307500000024F400B5
:10271800240000200000000000000000000000006D
:1027280000000000000000000000000000000000A1
:102738000000000000000000000000000000000091
:102748000000000000000000000000000000000081
:102758000000000000000000000000000000000071
:102768000000000000000000000000000000000061
:10277800000000004300000000000000000000000E
:102788000000000000000000000000000000000041
:1027980000000000430000000000000000000000EE
:1027A8000000000000000000000000000000000021
:1027B80000000000430000000000000000000000CE
:1027C8000000000000000000000000000000000001
:1027D80000000000430000000000000000000000AE
:1027E80000000000000000000000000000000000E1
:1027F800000000004300000000000000000000008E
:1028080000000000000000000000000000000000C0
:10281800000000004300000000000000000000006D
:1028280000000000000000000000000000000000A0
:10283800000000004300000000000000000000004D
:102848000000000000000000000000000000000080
:10285800000000006F2500084B250008000000005C
:10286800E7250008E5250008E6250008E625000814
:10287800E6250008E6250008E6250008E625000804
:10288800E6250008E6250008E6250008FFFFFFFF0B
:10289800FFFFFFFFFFFFFFFFFFFF000001004153A5
:1028A800434949000000000000000000000000004B
:1028B800000000000000000000000000000041537C
:1028C800434949000000000000000000000000002B
:1028D80000000000000000000000000000000000F0
:04000005080022BD10
:00000001FF
